:10000000600D0020ED170000B34000004118000013
:1000100041180000411800004118000000000000D5
:100020000000000000000000000000000D160000AD
:100030004118000000000000B915000093400000C6
:10004000AD170000AD170000AD170000AD170000A0
:10005000AD170000AD170000AD170000AD17000090
:10006000AD170000AD170000AD170000AD17000080
:10007000AD170000AD170000AD170000AD17000070
:10008000AD170000AD170000AD170000AD17000060
:10009000AD170000AD170000AD170000AD17000050
:1000A000AD170000AD170000AD170000AD17000040
:1000B000AD170000AD170000AD170000AD17000030
:1000C000AD170000AD170000AD170000AD17000020
:1000D000AD170000AD170000AD170000AD17000010
:1000E000AD170000AD170000AD170000AD17000000
:1000F000AD170000AD170000AD170000AD170000F0
:1001000053B94AB9002908BF00281CBF4FF0FF317E
:100110004FF0FF3000F06CB9ADF1080C6DE904CE82
:1001200000F006F8DDF804E0DDE9022304B07047D2
:100130002DE9F047089E0D4604468E46002B40F000
:1001400082808A42174646D9B2FA82F24AB1C2F197
:10015000200105FA02F320FA01F1974041EA030E6B
:1001600094404FEA1748230CBEFBF8FCB9B208FBD9
:100170001CEE43EA0E430CFB01F098420AD9FB182F
:100180000CF1FF3580F01681984240F21381ACF1FA
:10019000020C3B441B1AA4B2B3FBF8F008FB10336B
:1001A00044EA034400FB01F1A14209D93C1900F1E2
:1001B000FF3380F00181A14240F2FE8002383C44CE
:1001C000641A40EA0C4000211EB1D4400023C6E965
:1001D0000043BDE8F08702B9FFDEB2FA82F2002ADE
:1001E0004FD1CB1B4FEA174E1FFA87F80121B3FB03
:1001F000FEFC250C0EFB1C3345EA034508FB0CF303
:10020000AB4207D97D190CF1FF3002D2AB4200F2AC
:10021000E7808446ED1AA3B2B5FBFEF00EFB105545
:1002200043EA054408FB00F8A04507D93C1900F152
:10023000FF3302D2A04500F2D7801846A4EB080491
:1002400040EA0C40C0E78B4208D9002E00F0AF8096
:100250000021C6E900050846BDE8F087B3FA83F13E
:1002600000294BD1AB4202D3824200F2B780841AFC
:1002700065EB030301209E46002EAAD0C6E9004E7E
:10028000A7E7C2F1200C01FA02F3974020FA0CF024
:100290004FEA174E21FA0CFC1843BCFBFEF1050C8B
:1002A0000EFB11CC1FFA87F845EA0C4501FB08F359
:1002B000AB4204FA02F409D97D1901F1FF3C80F048
:1002C0008B80AB4240F2888002393D44EB1A85B204
:1002D000B3FBFEF00EFB103345EA034500FB08F3C9
:1002E000AB4207D97D1900F1FF3C71D2AB426FD907
:1002F00002383D44EB1A40EA014178E7C1F1200C95
:100300008B4022FA0CF71F4320FA0CF405FA01F394
:100310004FEA174E25FA0CF51C43230CB5FBFEF9EA
:100320001FFA87F80EFB195543EA054509FB08FA41
:10033000AA4502FA01F200FA01F308D97D1909F180
:10034000FF3047D2AA4545D9A9F102093D44A5EBA2
:100350000A05A4B2B5FBFEF00EFB105544EA0544B5
:1003600000FB08F8A04507D93C1900F1FF352DD254
:10037000A0452BD902383C4440EA0940A4EB0804CC
:10038000A0FB02894C45C6464D4619D316D05EB136
:10039000B3EB0E0264EB050404FA0CFCCA404CEA11
:1003A0000202CC40C6E900240021BDE8F0873146B6
:1003B00030460EE7AC46EDE6184601E74345E6D287
:1003C000B8EB020E69EB07050138E0E72846D3E7F2
:1003D00060468FE78146BAE7614677E708464BE714
:1003E000ACF1020C3D4415E702383C4426E700BF5F
:1003F000704700BF0149024803F08EBC284B000043
:100400003B4B00000B6801330B60014B1B68184726
:1004100000000020014B1860704700BF0000002062
:1004200007B50B46002102460191034801A900F0DF
:10043000EBF803B05DF804FB050400002DE9F84F6C
:10044000B0F8189019F00808044693460DD0012919
:100450000CBF49F0100949F02009A0F818908BF35F
:100460001188BFF36F8FBDE8F88F09F007090229E3
:1004700007D1204603F05DFC0028F0D00128238B33
:1004800050D16769218B002F15DA256821F007010B
:10049000C4E9008841F0010121830026218B01F08D
:1004A000070ACA4502D0A368002B5CD10DB9002E03
:1004B00074D0002358E001F007035A1F012A20D806
:1004C00021F00701062B256889B2C4E900880CD108
:1004D000002D2B4638BF00232BB1628B1B680132E5
:1004E0006283002BF8D141F002012183204603F002
:1004F00020FC06460028D1D0238B43F02003238321
:10050000CBE7042B0CD121F0070189B221832046CF
:1005100003F00FFC05460028BFD041F020012183E5
:100520000025BAE7032809D1226923F007031668DA
:1005300043F00603238300252F46AFE7042806D1A6
:10054000226923F00703566843F00403F2E7052805
:1005500006D1226923F00703966843F00503E9E713
:1005600000252E46E8E7012341F0080121838BF3A3
:100570001188BFF36F8F03BB002D33D116B1214912
:100580002046B0474FF02003EFF3118B83F311881F
:10059000BFF36F8F238B23F008032383238BDA06AB
:1005A00028D523F0100323830121B4F8189009F013
:1005B000070900297FF45BAF51E7A1680029DBD070
:1005C0000B68D1F804B0002B38BF0023994652467F
:1005D0003B462046D847B9F1000FCDD0D9F80030BE
:1005E0004946EEE729463B46524620462D6803F031
:1005F000BCFBC1E713F020011EBF23F020032383BF
:100600000221D2E7973D00002DE9F04F91B08B46D3
:10061000029092461C4600259AF8000008B9284628
:100620005EE325280AF1010707D0029B5946984747
:100630000028C0F25583013510E2182200210AA8D3
:1006400003F085FD9AF80130252B78D000229446DE
:10065000164696461046394617F8013B2B2B00F0FC
:100660009D8000F29480202B00F09B80232B00F0D3
:100670009A8028B19DF8300040F004008DF83000D9
:10068000BEF1000F05D09DF8300040F008008DF855
:1006900030002EB19DF8300040F010008DF8300091
:1006A000BCF1000F05D09DF8300040F020008DF81F
:1006B00030002AB19DF8302042F040028DF8302001
:1006C0009DF8302002F04400442803D16FF38612D5
:1006D0008DF830209DF830202A2B42F080028DF8D2
:1006E00030207BD19DF8312042F001024B1C8DF867
:1006F00031201A782E2A9DF831200CBF01210021CB
:1007000061F341028DF8312074D15A782A2A6AD0D7
:10071000013300210A26184610F8012BA2F13007F8
:10072000092F40F28E809DF830200E91C2F34000D8
:1007300040EAD17161F341028DF830205AE00AF1AC
:1007400002078DF833309DF83130D90740F14981E7
:1007500054F8049BB9F1000F07DA9DF8302042F0FD
:1007600004028DF83020C9F100095A0740F1428196
:1007700054F8048BB8F1000F80F241819DF83130BC
:100780006FF341038DF831304FF0FF3837E12D2BF7
:100790000CD0302B7FF46DAF01225CE74FF0010EDF
:1007A00059E7012657E74FF0010C54E7012052E7C3
:1007B0000CFB0202303A33461E4616F8010BA0F13C
:1007C0003007092FF4D9994293D09DF830100D923B
:1007D000D20F62F341018DF830108AE70B460022F8
:1007E0004FF00A0CE8E79DF8312042F004028DF842
:1007F000312002331F4617F8012B6C2A41D025D82F
:10080000682A2BD06A2A46D04C2A4CD01F4617F8AB
:10081000012B9DF831308DF83320782A00F2D980F1
:10082000572A4DD8412A03D0453A022A00F2D180F6
:100830009DF83230042262F302038DF83230012336
:100840009EE006FB01213039034664E7742A26D076
:100850007A2ADBD19DF8313006220DE05A78682AD9
:100860009DF8312006D1012161F3C6028DF83120B7
:100870009F1CCCE71346022262F3C6038DF8313089
:10088000C5E75A786C2A9DF8312001D10421EBE7A5
:1008900013460322F0E79DF831300522ECE79DF87E
:1008A00031300722E8E7BDF8303023F4F04323F07D
:1008B000020343F4804343F00203ADF83030A6E76F
:1008C000A2F15801202900F2848001A050F821F003
:1008D00095090000D3090000D3090000D3090000E6
:1008E000D3090000D3090000D3090000D309000098
:1008F000D309000031080000D30900009509000069
:1009000055090000310800003108000031080000DE
:10091000D309000055090000D3090000D3090000E5
:10092000D3090000D30900009D09000095090000CB
:10093000B9090000D3090000D3090000B90900007B
:10094000D309000095090000D3090000D309000075
:10095000950900009DF83210012003F0780360F340
:100960000201402B8DF8321002BF9DF8301041F08B
:1009700001018DF83010632A31D1003B18BF0123EB
:100980009DF83020C2F340010B4363F341028DF820
:100990003020D8E69DF832100220DEE79DF83220A4
:1009A00003F07803A3F14000032161F30202434204
:1009B0008DF832204341E3E79DF83220032113F004
:1009C000780F61F302028DF8322014BF0123002357
:1009D000D6E79DF8303043F001038DF83030002326
:1009E000CEE79DF93020002AB4BFDDF834904FF0F7
:1009F000FF39BAE69B077FF5C7AEDDF838809DF872
:100A000031200023CDE90D339DF8323003F0070388
:100A1000012BC2F3C30236D1D31E042B20D8DFE84A
:100A200003F00307071F1F0054F8040BC11704E06D
:100A3000073424F00704F4E80201CDE90A019DF827
:100A4000303013F0030654D002983B4652465946C4
:100A500003F06FFA0028C0F243810544BA46DBE593
:100A600054F8040B012A4FEAE071CDE90A0105D1DF
:100A70009DF828300A9300230B93E0E7022ADED189
:100A8000BDF92800D2E7022B23D1D31E042B13D8A3
:100A9000DFE803F0030A0A12120020680A9000211E
:100AA000231D0B911C46CAE7073424F00703F3E823
:100AB0000201CDE90A01F5E754F8043B0A93012A43
:100AC0004FF000030B93D3D0022AB8D1BDF82830E1
:100AD000D0E7042B07D1073424F00704F4E802011F
:100AE000CDE90A01ABE7032B04BF54F8043B0A939A
:100AF000A5E79DF833007828B0D8622822D82528A9
:100B00003FF493AD5828A9D10DF126030093DDE9F8
:100B10000A0104AB0CAA03F0C1F98246B8F1000F38
:100B20000DF126000CDB9DF83020A0EB0A036FF3DB
:100B3000861298458DF8302002D9A8EB03030D9357
:100B400080463DE06338152888D801A151F820F08F
:100B5000D10B0000350C00005D0A00005D0A0000AA
:100B60005D0A00005D0A0000350C00005D0A00000F
:100B70005D0A00005D0A00005D0A0000930C0000A1
:100B8000610C0000650C00005D0A00005D0A0000B9
:100B9000A90B00005D0A0000610C00005D0A000066
:100BA0005D0A0000610C0000B8F1000FDDF828A01C
:100BB0000ADB4146504603F08AFA0AEB0008002699
:100BC000BAF1000F0CD149E7504603F079FAF4E787
:100BD0000A9B8DF8103000260DF111080DF1100A56
:100BE000A8EB0A0306B101339DF83220D0066BD57D
:100BF000023352060D9948BF0E9A0B4448BF9B180A
:100C0000B9F1000F79DD9DF83020A9EB0309C2F39B
:100C100080030393530770D4500664D546B1029BFA
:100C200059463046984700285ADB039B01351E463B
:100C3000302359E01E0711D413F0100618BF2026E8
:100C4000DDE90A23002A73F10001BFF65DAF5242CD
:100C500063EB4303CDE90A232D2655E72B26EFE767
:100C6000002651E70A9848B30DF1260300930CAA19
:100C700004AB002103F012F9BDF8323003F0EF03AA
:100C800043F4F04343F010038246ADF832300026BF
:100C900044E70A9B072A3FF6E1AEDFE802F00D04C5
:100CA000060D08080D0D1D70D8E61D80D6E62846F5
:100CB000E917C3E90001D1E61D60CFE6DFF8C48083
:100CC0000646A8F1050A8BE7110748BF013390E7F4
:100CD000184603935946029B98470028039B04DA61
:100CE00011B0BDE8F08F20234D444A46002AA5EB01
:100CF000090109F1FF39EBDC0D4636B1029B59467B
:100D0000304698470028EBDB01359DF83230D90694
:100D100001D41A0706D5029B59463020984700286F
:100D2000DEDB01359DF83230DB0607D59DF8330058
:100D3000029B594698470028D2DB01350D9E2E4470
:100D4000731B002B16DC029843465246594603F0AB
:100D5000F0F80028C4DB0544A944A9EB0503002BE7
:100D60007FF77CAE029B5946202098470028B7DBCE
:100D70000135F2E7029B5946302098470028AFDB47
:100D80000135DDE7514B000008B504464FF0200265
:100D9000EFF3118382F31188BFF36F8F03F07BF9B8
:100DA000204600F083FF034802F0B6FF00F0C6FCC7
:100DB000FCE700BF524B0000F8B505464FF020039A
:100DC000EFF3118683F31188BFF36F8F0B4B1C6811
:100DD000002C38BF00245CB1094FD4E90132002D4A
:100DE00008BF13460BB1387898472468002CF4D11B
:100DF00086F31188BFF36F8FF8BD00BF800200201B
:100E000088020020084B10B51C685CB901221A60EA
:100E1000064B93E8070003F0D5F92046BDE81040E3
:100E2000FFF7CABF10BD00BF0400002088020020E9
:100E3000F0B585B06E4601460546304603F090F8A1
:100E400096E80700144C84E80700207808B3134B99
:100E5000002119606B1C0ED0114817464FF4004654
:100E60000021104A0023E6FB0701FFF749F90121A1
:100E7000281A03F021FC02F0E3F80120FFF79CFFA1
:100E800094E8070003F08BF9FFF7BCFF02F0CAF902
:100E9000207805B0F0BD00BF8802002004000020CB
:100EA0003F420F0040420F0010B50748074C01F0C9
:100EB00095FD074B1860204600F0DAFE2046FFF74C
:100EC000A9FA002010BD00BF7B4B0000D50E00002A
:100ED000940200200A2838B5074D044604D128683A
:100EE00083680D215B68984728688368E1B25B6876
:100EF0009847204638BD00BF940200200E4A70B5C6
:100F0000841AA3100D4C5C430546E4B20C2000FB90
:100F100004200E464021084403F030F8011E05DB92
:100F2000074B03EBC4046368984700212846334607
:100F3000BDE87040184700BFAC020020B76DDBB6BB
:100F40003C4900002DE9F041104E841BA310104CC9
:100F50005C43E4B20C256543804605F140000F4632
:100F60003044402103F023F8011E09DB094A7319BC
:100F7000C3E90E27084B53F83430BDE8F041184759
:100F800040463B46BDE8F041184700BFAC02002098
:100F9000B76DDBB6114000003C490000002270B57F
:100FA00001210446104600F05FFB002000F03EFBEC
:100FB0000F4801F0A9FB0F4B984215D103F026FA18
:100FC00026690D49304602F003FF00280BDB01259E
:100FD00035642469084904F11C0002F0F9FE002878
:100FE00001DBE564002070BD6FF00400FBE700BF8B
:100FF000311000000000AD0B4C49000001460C23ED
:1010000009484B4370B5C418D4E90E56002240334A
:10101000A263184402F0E9FF2DB132462B46034883
:10102000BDE87040184770BDAC020020AC00002045
:1010300010B1012804D07047034B1B6C5B0701D132
:10104000FFF7DCBF704700BFAC02002008B54FF0CF
:101050002003EFF3118183F31188BFF36F8F124ADE
:10106000136843F0020013F0010310600CD04FF03E
:101070008042D2F80C34D2F80C2413F0010303D0D0
:101080000A4802F0B2FF012381F31188BFF36F8F8A
:1010900023B1BDE808400020FFF7B0BFBDE808401D
:1010A000012001F041BB00BFFC020020EC02002047
:1010B000094BBFF35B8F53E8002F22F0020143E896
:1010C00000100028F7D1BFF35B8FD30702D40120B3
:1010D00001F05CBB704700BFFC0200201FB500227E
:1010E0000123CDE90223094ACDF800D06B46CDF8A3
:1010F00004D002F0B3FF002805DB4FF48042002348
:10110000684601F019FF05B05DF804FB2F400000B0
:101110002DE9F8433A49BFF35B8F0646012251E8B7
:10112000003F41E800200028F9D1BFF35B8F33B9BD
:10113000344935484B60CB608A6002F05CFE731E18
:10114000012B32D8012E07D14FF08043D3F81C3445
:1011500003F00303012B28D003F0CBF9044618B9A0
:101160002A4B1B78002B44D14FF02003EFF311855D
:1011700083F31188BFF36F8F0124254FDFF894802C
:10118000DFF894904FF08042D2F81834D2F8182447
:10119000D2030CD503F00303012B01D0012E06D19D
:1011A0000CB385F31188BFF36F8FBDE8F883ACB142
:1011B000284600F0D1FA4FF08042D2F81835002BC3
:1011C000E0D139680029DDD03B603B680123C2F8DB
:1011D0001835C8F88031C9F80030D3E70021212044
:1011E00002F0BCF9E7E74FF080430222C3F8042382
:1011F000DBE74FF080430222C3F808230546BCE733
:10120000000300209C020020C80200204A090020A0
:101210000401004000E100E008000040044A1368B7
:10122000C81A20F07F400344136002F003BB00BFE4
:10123000140300202DE9F047860006F1804600F1F6
:10124000500406F58836A400DFF87C80D6F84035D7
:10125000A4B204F180444FF4803721F07F4504F5B7
:1012600088348740C146D8F804A5A3EB0A0323F0CD
:101270007F432AF07F42012BC6F8402502D113207C
:1012800003F038FA0AF10202AB1A23F07F43B3F5F8
:10129000000F88BF1546002323602368C9F84473F4
:1012A00025F07F43C6F84035D9F804359A4506D075
:1012B000EB1A023B23F07F43B3F5000F01D8BDE8E2
:1012C000F0872B46CFE700BF00100140F8B5104E65
:1012D000104F0025104B00201C681A4605B1F8BDC0
:1012E000D6F80413C903FAD539680029F7D03D6050
:1012F00039684FF48031C6F84813D6F840150125F7
:101300001CB15A681860A047E4E71460E7E700BF23
:1013100000100140401101400803002038B5104D75
:1013200000244FF48033C5F80845C5F804330D4B4D
:101330004FF40032C3F8802101212246112000F031
:1013400093F9112000F072F9074A01231360074A4C
:101350002B6002201360FFF7DBFE204638BD00BF84
:101360000010014000E100E00810014010030020DF
:10137000134BB0F1FF3F08BF1846013800281CDDB1
:101380009842A8BF18460F4BD3F804250E4B196896
:10139000521A12F4000F22F07F4318BF00200B4AAC
:1013A000013303440A48106000205060044A93420D
:1013B00094BFC9188918FFF73DBF0020E3E700BFBD
:1013C000FFFF7F00001001401403002008030020ED
:1013D0001D120000044BD3F80405044B1B68C01A0F
:1013E00020F07F40704700BF001001401403002030
:1013F000014802F0FFBA00BF5849000008B5D0B15B
:101400004368042B11D100220368BFF35B8F53E8BC
:10141000001F012903D143E800200028F7D1BFF3C2
:101420005B8F074808BF104608BD3BB1006801F05C
:101430001DFD0020F8E76FF4E040F5E70148F3E711
:10144000E98FFFFFEA8FFFFF10B5044618B90D4B77
:101450000D485B689847616808290DD031F0040396
:101460000AD011F0020108D00848214603F018F80C
:10147000002323600023636010BD2068142202F063
:1014800066FEF7E74C000020924B00001803002096
:1014900010B5044618B9164B16485B689847636840
:1014A000042B23D0082B21D0CBB92368BBB9124819
:1014B0004FF0FF324FF0FF33214601F089FB08B9AE
:1014C00023681BB90A4B0D485B68984720681422B3
:1014D000002102F03CFE636843F002036360206871
:1014E00003F014F8636843F00103636010BD00BFAC
:1014F0004C000020924B000018030020B84B000065
:1015000008B508B34368042B10D101220368BFF368
:101510005B8F53E8001F002903D143E80020002817
:10152000F7D1BFF35B8F0BD1002008BD53B100682A
:101530004FF0FF324FF0FF3301F020FC0028F3D0D2
:101540000348F2E70348F0E76FF4E040EDE700BF3F
:10155000E98FFFFFEA8FFFFF08B5064906484023E1
:10156000142202F082FFBDE808400449044802F05A
:1015700097BA00BF34030020180300207049000010
:1015800060490000094A0A4993680968996709494E
:1015900058674B6843F080534B60002383F31188F6
:1015A000BFF36F8F9368986F704700BFF0080020FB
:1015B0009C4A000000ED00E012498A684FF03000BC
:1015C0001044EFF3098C80E8F01F202080F311888D
:1015D000BFF36F8F0C4F4FF000664A6A8A603E601F
:1015E000506F0023536780F3118804B5104600F054
:1015F0008FFABDE8044002F1300090E8F01F8CF350
:1016000009887047F008002004ED00E01EF0040F88
:101610000CBFEFF30880EFF30980816911F8021C19
:101620000229FFD001B502F040FD01BD43B2002BFD
:1016300008DB012200F01F0002FA00F05B09024AF9
:1016400042F82300704700BF00E100E0054B42096B
:1016500000F01F0053F82220012303FA00F010408D
:10166000704700BF00E100E043B2002BA8BF03F1C8
:10167000604301F10101B8BF064B4FEA4111ACBF15
:1016800003F5614300F00F00C9B2B4BF195483F8E9
:101690000013704714ED00E042F8203C009B42F834
:1016A0001C3C0A49019B42F8183C029B42F8143C3E
:1016B00021F001014FF0807342F8043C42F8081C0D
:1016C0000023203A02654367704700BF893E00004F
:1016D0000B4A0346906890B113F1160F406E05D087
:1016E000A0F120029A4206D8834204D281422CBF44
:1016F0000021012100E00021002908BF00207047DF
:10170000F008002008B5094B98600D46144600F01B
:10171000FFF9204685F30988002163B681F311881B
:10172000BFF36F8F0022002302F0AEFBF008002011
:10173000014910220A60704710ED00E072B6404087
:1017400080F31188BFF36F8FBFF34F8F30BF62B646
:10175000BFF36F8F704700BF72B6494081F31188A5
:1017600020BF80F3118862B6704700BF30BFFFF71B
:10177000FDBF00BF0B4A08B50B4B22F07F029A60F9
:10178000BFF34F8FBFF36F8FD3F8882022F470021E
:10179000C3F8882001F04EF901F05AFF00F08EF9ED
:1017A00001F06CF90000000000ED00E001B572B638
:1017B0000B4A106A00281EBF0021116202F09FFE32
:1017C00062B6EFF30580A0F110004FEAC0000549B2
:1017D000014409C99847BDE8014003490847000092
:1017E000F0080020684700001D1A0000002080F368
:1017F0001488BFF36F8F02F0D0FC00200D49086001
:10180000BFF34F8F0C4880F3088800F025F92020A3
:1018100080F3118809484FF40261401880F3098869
:10182000EFF314800221084380F31488BFF36F8F15
:10183000FFF7A0FF94ED00E0600D0020E00E002017
:10184000EFF30880EFF3098101B5724600F068F804
:1018500001BD00BF38B5194B14469A6A9A6A9A6A54
:101860000546900719D5586B9A6A120615D519B115
:101870009A6A22F080029A629A6A9A6A9A6AD106F1
:101880000ED49B6A9A070BD400200C4A936A43F04B
:10189000FF0393620023237038BD6FF01500EBE760
:1018A000064B5B681B05EFD52946FFF711FF0028A3
:1018B000EAD080F309880220E7E700BF00ED00E0EE
:1018C0000D4B9A6A9A6A9A6A920508D59A6B9A6A37
:1018D000120404D518B19A6A22F400429A62064BA7
:1018E0009A6A9A6AD20558BF9A6A9A6A002042F4A4
:1018F0007F429A620870704700ED00E0074B9A6AD9
:101900009A6A9A6A9A6A9A6A9A6A9A6A6FEA024222
:101910006FEA12429A620020704700BF00ED00E0BB
:1019200070B5374B5B688AB00E46C3F308030025D9
:1019300085F31188BFF36F8F02F07F41B1F17F4FC4
:1019400011D102F00C0108290DD0110701D406466F
:1019500001250022033B8DF80720032B48D8DFE840
:1019600003F0043F433C2E46F3E7254BDA6A920727
:101970003ED4DC6A14F0804409D028331B78F3B1DC
:101980000DF1070201213046FFF764FF04469DF880
:10199000073093B92022314602A802F0ADFB099B23
:1019A00045B3C3F3080222B96FEA53236FEA432316
:1019B000099302A9204602F076FB0AB070BD114BD4
:1019C0001B782BB10DF107010120FFF779FFDDE74F
:1019D0000D4B188884B2002CD9D0FFF78FFFD5E7C4
:1019E0000DF107020021CEE70DF107010020ECE721
:1019F0000024CCE723F4FF7323F00103D8E700BFF2
:101A000000ED00E029ED00E02AED00E0024A536914
:101A100043F010035361704700ED00E0044B9968F8
:101A2000586A884203D003494FF080520A607047D9
:101A3000F008002004ED00E0064A11680023C1F31D
:101A4000072118468B4200D1704793601061013323
:101A5000F8E700BF90ED00E008B572B6002383F30D
:101A60001388FFF7E9FF144B4FF0FF32C3F88020D3
:101A7000C3F88420C3F88820C3F88C20C3F89020D2
:101A8000C3F89420C3F89820C3F89C20C3F88021A1
:101A9000C3F88421C3F88821C3F88C21C3F89021AE
:101AA000C3F89421C3F89821C3F89C2162B6BFF310
:101AB0004F8FBFF36F8F08BD00E100E004480023A3
:101AC0002021C2180133302B82F80013F9D170475E
:101AD00000E100E0064B9B68834207D1EFF30583EA
:101AE00023B1044A536843F08053536001F05EBD54
:101AF000F008002000ED00E0024B034A03480121FA
:101B000000F068B8000004200000002084490000B4
:101B1000426E054B203A1A60044A2021C3E90112A3
:101B20001846012100F060B83408002000000B15B1
:101B3000F0B51E4F00268E4201DB1046F0BD446812
:101B400084B353B104F1FF3C14EA0C0F18D11F2CDD
:101B500016D905681CEA050F12D1202C0568D0F8AB
:101B600008C0D2B20FD9B4F1004F0ED8013CB4FA7C
:101B700084F4C4F11F046400072A4CEA040406D963
:101B80006FF01502D9E70824F6E73E24F4E725F0C4
:101B90001F05154345F0100544F00104BA60FD60CF
:101BA00001323C6101360C30C5E700BF90ED00E02A
:101BB000034B05225A60BFF34F8FBFF36F8F7047FF
:101BC00090ED00E0BFF35F8F014B00225A60704739
:101BD00090ED00E010B5034C01232278FFF7A8FF39
:101BE000207010BD4809002008B5084A002312786B
:101BF000FFF79EFF10F1160F03D0054B00220728B8
:101C000000DD08BD98601A610130F8E7480900203E
:101C100090ED00E013490868082810B51ED8FFF7BA
:101C2000D1FF114C49680022904201F10C0105D10D
:101C30000E4B1870FFF7BCFF002010BDA26051F8DA
:101C40000C3C23F01F03134343F01003E36051F8EF
:101C5000043C43F0010323610132E5E74FF0FF301C
:101C6000EBE700BF9049000090ED00E0480900203C
:101C7000014B1860704700BF280000204FF0200380
:101C8000EFF3118283F31188BFF36F8F06490123AD
:101C9000C1F840354FF08041C1F8783582F31188A2
:101CA000BFF36F8F0020704700E001404FF080438A
:101CB000C0B2C3F81C05BFF34F8F0549054BCA6876
:101CC00002F4E0621343CB60BFF34F8F00BFFDE728
:101CD00000ED00E00400FA0520B1034B800143F061
:101CE00001031847704700BF204900002DE9F0416B
:101CF0001A4D002701266C79D5F80080404602F085
:101D000090FB40B3AB792979002B14BF4FF4D0532B
:101D10004FF4B0532343D8F81040D8F808E02068B7
:101D2000DA0748BF83F4406323F4805206FA01FCCB
:101D3000DB074CBF4CEA000020EA0C002060DEF814
:101D400000304046984720B90137102F05F10805AB
:101D5000D1D1BDE8F0816FF01200FAE7B049000080
:101D600008B5094B1A786AB90121197006200521B6
:101D7000FFF77AFC0620FFF759FC044B4FF00042B6
:101D8000C3F80423002008BD49090020006000407A
:101D90002B4BF0B544682B481340834241D00DD8FB
:101DA000062B15D005D89BB1022B3CD06FF0150047
:101DB00036E0B3F5801FF9D1012309E022488342C0
:101DC00033D0B3F5A00F32D0B3F5800FEED102239C
:101DD000D00654BFC2F34016032682F480759705DF
:101DE000C2F34020C5F3002507D512F4006F6768E1
:101DF0001FD001228A40C7F80825227A134C012AF5
:101E000001F01F0140EA450218BF4FF0A04442EA2A
:101E1000032301F5E07143EA860344F821300020F2
:101E2000F0BD0723D4E70423D2E70523D0E703233B
:101E3000CEE7520542BF01228A40C7F80C25DCE7F5
:101E40000600F000060010000200400000030050F1
:101E500000F01F024009084B012818BF4FF0A043B3
:101E600003EB8203D3F8002722F4403242EA014216
:101E7000C3F80027704700BF000300502DE9F84F5A
:101E80000369D0F804A0DE68DFF87CB08846D3E9A7
:101E900005210A4326EA0206DAF804201B69D2F873
:101EA00010555D4026EA0505374601244FF000092C
:101EB00017B92846BDE8F88F3C4221D09AF808307F
:101EC00009F01F00344240EA431014D14209012AAC
:101ED00000F01F0314BF4FF0A0425A4603F5E07311
:101EE00052F82330C3F30143022B02BFD8F800306D
:101EF0002343C8F800300021FFF7AAFF27EA0407B0
:101F000009F101096400D3E700030050F7B50E465C
:101F100041680769097A06F01F05B2F5A03F45EA56
:101F2000411510D16809012805F01F015D4801F530
:101F3000E07118BF4FF0A04050F82110C80707D536
:101F40006FF0850093E0B2F5005FF96800F09180D2
:101F5000F8680121B14001437869F9600121B1407D
:101F6000B2F5A03FBA690CBF08438843B3F5C02F50
:101F70000CBF0A438A43BA613A697861B3F5802F8E
:101F80000CBF114322EA0101474A3961D2F80433F8
:101F90000020DBB200F5A27152F82110C1F3052137
:101FA0008D426BD123FA00F1C90767D5830003F195
:101FB000804303F5C043D3F8101521F00101C3F8A5
:101FC000101501238340C2F80833C0B200F058FC5A
:101FD00028460021FFF73CFFF868F04010F00100B0
:101FE00045D07869F04010F001044ED0BB69F34051
:101FF000DB075FBF396921FA06F606F00106C6F174
:1020000002060DF1070054BFF6B2032600F05AFC99
:10201000264B984236D19DF807108B0003F1804380
:1020200003F5C0432D02D3F8102522F44F3222F4D9
:102030004072C3F81025D3F8102505F47C551543DC
:102040008A0002F1804202F5C24245EA06460020BB
:10205000C3F8106510601268D3F8102542F0010231
:10206000C3F81025104A01238B40C2F8043303B093
:10207000F0BD0120B04021EA00016DE701300828E1
:1020800088D1A5E76FF01200F1E73969F14001F05E
:102090000101C1F103012846C9B2FFF7D9FE20466C
:1020A000E5E700BF00030050006000400000AD0BFA
:1020B000F0B5002485B0CDE90044CDE90244264EB8
:1020C00035685DB102A92548FFF7D8FE03A9009045
:1020D0002348FFF7D3FE019034603368214C00227F
:1020E00001269446D4F8043306FA02F119421BD0B3
:1020F000910001F1804101F5C2410B68A3B102F5E5
:10210000A27304AF54F82330C1F800C0C3F34030C9
:1021100007EB8000C3F3042350F8107C06FA03F3A6
:102120003B4340F8103C0B680132082ADAD1009A90
:102130001AB10A490C4802F05BF8019A1AB1084931
:102140000A4802F055F82DB1044802F0BBF80448E3
:1021500002F0B8F805B0F0BD7C610040F40000204A
:102160000C010020006000404C080020680800209E
:10217000F0B54B79012B2AD0032B25D110268B7972
:10218000032B21D1CC792CB1012C1DD143685B6884
:102190009B0719D00A7912B1022A15D10E220B68B9
:1021A0004568B3F5164F2D6865D02DD8B3F5165F89
:1021B00064D016D8B3F5966F62D00AD8B3F5967F7F
:1021C00061D0B3F5167F61D06FF0850052E0002634
:1021D000D5E7B3F5166F5CD0B3F5965FF4D1374B06
:1021E0003CE0B3F5E14F57D007D8B3F5615F55D068
:1021F000B3F5964FE8D1324B30E047F61227BB4299
:10220000E2D14FF4000329E0B3F5613F48D013D881
:10221000B3F5963F47D009D84DF6C027BB4244D00E
:10222000B3F5614FD0D14FF46B0317E0B3F5E13F45
:10223000CAD14FF0EB7311E0B3F5612F38D008D855
:10224000204FBB4237D0B3F5E12FBDD14FF0E8634B
:1022500004E01D4FBB42B7D14FF08053C5F8243581
:10226000036903C9344322430433C5F86C2583E86A
:1022700003000020F0BD4FF41D03EFE7134BEDE723
:102280004FF49E23EAE74FF4A033E7E74FF41C3303
:10229000E4E74FF41D23E1E70D4BDFE70D4BDDE7EE
:1022A0004FF06C73DAE70C4BD8E74FF46503D5E7D2
:1022B0004FF07063D2E74FF08063CFE700B01300B8
:1022C00000A04E0090D0030040420F0000502700B5
:1022D00000C0750000F03A0000903A01F8B50669B8
:1022E00005460F4602F005F910B92C4B1B7883B94F
:1022F0004FF02003EFF3118483F31188BFF36F8F46
:10230000284602F04EF828BB84F31188BFF36F8F84
:10231000EEE76424284602F044F870B9012002F088
:1023200073F8013CF6D10021212001F017F9F0E704
:1023300084F31188BFF36F8FF5E74FF02003EFF3BD
:10234000118483F31188BFF36F8F284602F029F8B8
:102350000028EDD006F8107F69680B680122C3F8E9
:102360004465C3F848250022C3F82021D3F8200192
:10237000C3F85821D3F858214A68D20641BF082231
:10238000C3F800254FF48002C3F8042301229A60A9
:1023900084F31188BFF36F8FF8BD00BF4A09002096
:1023A00000F01F0240090128044B02F5E07218BF3B
:1023B0004FF0A043032143F8221070470003005060
:1023C00000F01F0140090128044B4FF0010218BF23
:1023D0004FF0A0438A40C3F808257047000300501F
:1023E000F8B50022054601210220FFF73DF9022041
:1023F000FFF71CF96B682E691C680023C4F80035D0
:1024000005203560FFF7DCFF0520FFF7C9FF4FF01F
:10241000A0430C220521C3F80C27C4F80C15032196
:10242000C4F814152820C3F81C27FFF7C9FF28207B
:10243000FFF7B6FF29692823C4F808350723C4F835
:10244000103504312846FFF793FE0746002844D193
:102450006B685B68190719D506F1120000F06AFA7B
:10246000204B98423BD1B07CC30003F1804303F57D
:10247000F83304F10C0204F59071C3F81015C3F899
:102480001425194A01238340C2F804350823C4F8EF
:1024900000350023C4F81031D4F8103106F11103CF
:1024A000C4F834350123C4F8383523606B685B68A1
:1024B0001A075CBF4FF48072C4F80423DB0644BFE4
:1024C0004FF48003C4F8043310360023C4F8446585
:1024D000C4F848350123A360E3603846F8BD6FF0C7
:1024E0000407FAE70000AD0B00F00140034B186849
:1024F000A0F1080358425841704700BF3001001056
:10250000064B1B68082B06D1054B1B68052B02D810
:10251000044AD05C70470020704700BF30010010B3
:1025200034010010084C0000024AD2F80034002B9D
:10253000FBD0704700E0014010B5FFF7D7FF40B176
:102540004FF080430022C3F80C21C3F81021C3F8D8
:102550003825FFF7CBFF002846D04FF080525B4B69
:10256000D2F80414C3F82015D2F80814C3F82415BF
:10257000D2F80C14C3F82815D2F81014C3F82C158F
:10258000D2F81414C3F83015D2F81814C3F834155F
:10259000D2F81C14C3F84015D2F82014C3F844151F
:1025A000D2F82414C3F84815D2F82814C3F84C15EF
:1025B000D2F82C14C3F85015D2F83014C3F85415BF
:1025C000D2F83414C3F86015D2F83814C3F864157F
:1025D000D2F83C14C3F86815D2F84014C3F86C154F
:1025E000D2F84424C3F87025FFF78AFF10B1384BA6
:1025F000384A1A60FFF784FF18B1374BFB22C3F843
:102600001825FFF77DFF48B13449354B0A681B6830
:1026100022F00F0203F00F0313430B60FFF770FF6C
:1026200018B1304B4FF400721A60FFF75FFF48B1EA
:102630004FF08043D3F80024D20744BF6FF001026B
:10264000C3F80024284B1B68082B0ED1274B1B68AE
:10265000052B02D8264AD35C3BB14FF01023D3F8A8
:1026600008224FF08043C3F858254FF01023D3F8C9
:102670000022002A03DBD3F80432002B22DA1D49A2
:102680000123C1F80435FFF74FFF4FF0102012244B
:10269000C0F80042FFF748FFC0F80442FFF744FFCC
:1026A0000023C1F80435FFF73FFFBFF34F8F1249F6
:1026B000124BCA6802F4E0621343CB60BFF34F8F42
:1026C00000BFFDE70E4B0F4A1A6010BD00C000406E
:1026D0008C5600404881030000F00040E40E0040AA
:1026E00058020010409602403001001034010010E2
:1026F000024C000000E0014000ED00E00400FA059B
:10270000400000200090D003044B1A7922B9012226
:1027100018609A8002487047024870478408002079
:102720000000AD0B0C00AD0B10B1012820D070479C
:102730004FF08043D3F81824D3F8181411F4803FD5
:10274000194611D002F00302012A0DD1C3F8182551
:102750000C4B00221A601B684FF080430222C3F822
:10276000042301229A6070470023C1F81835EFE76F
:10277000054B00221A601B684FF08043C3F8040326
:1027800018607047040100400001004038B510B1E6
:10279000012818D038BD4FF080430222C3F8082327
:1027A000184A10601268184A0121116042F210752F
:1027B0001C46D4F81834DB03ECD5012001F024FECC
:1027C000013DF6D1E6E7114B4FF080440022C4F8FA
:1027D00008031A601B680E4B42F210751860D4F89B
:1027E0000C34D4F80C24D20303F0010305D523B133
:1027F000012001F009FE013DF1D1064B00225A7182
:10280000C8E700BF040100400C0000400001004088
:102810000400004084080020164B1A6810B56AB105
:1028200000221A601B684FF080430122C3F808237E
:10283000114B587910B95A711B6898470F4B1A6899
:1028400072B100221A601B684FF08043D3F818243D
:10285000D3F81814920704D10122C3F818259A60FE
:1028600010BD0222C3F80823034BBDE810401B68CB
:1028700001201847000100408408002004010040A6
:10288000012303FA00F010F0FF0F12D04FF02003E5
:10289000EFF3118183F31188BFF36F8F064AD36D75
:1028A00023EA0000D06581F31188BFF36F8F0348DE
:1028B00070470348704700BF8C0800200000AD0B34
:1028C0000400AD0B2DE9F0410546DFF860E0164845
:1028D000DFF85C800024FF220126E3B24FF02001E4
:1028E000EFF3118C81F31188BFF36F8F22FA03F19C
:1028F000C9070AD5DEF85C1006FA03F7394201BFB2
:102900003943CEF85C1040462B708CF31188BFF32E
:102910006F8F404505D006FA03F39A4304F1010492
:10292000DBD1BDE8F08100BF0200AD0B8C080020B8
:102930000000AD0B2DE9F041144A154E154F054628
:10294000154800244FF0010E5FFA84FC4FF020037D
:10295000EFF3118883F31188BFF36F8F0EFA0CF336
:10296000134207D031680B4201BF1943316085F82B
:1029700000C0384688F31188BFF36F8FB84203D088
:102980009A4304F10104DFD1BDE8F081FFFF0F009D
:10299000EC0800200000AD0B0200AD0B0E4B70B533
:1029A00053F82040013053F82060A64200D870BD93
:1029B000D4E900352846984765B1EB6830B1002866
:1029C000B8BF4042FF28A8BFFF2018705A7842F0D5
:1029D00001025A700834E8E7884A000070B50546DD
:1029E00010B90024204670BD0378002BF9D00F4A9F
:1029F0000F4C1646944208D10D4CB442F1D02046FB
:102A000001F00FFD50B91834F7E7204601F009FD39
:102A100010B12368AB42E5D01834EBE721682846B3
:102A200001F05EFB0028EED1DCE700BF24010020AE
:102A3000AC0000200248034A0021121A01F087BBB3
:102A4000780100204C09002008B50A4B0122022021
:102A50001A70FFF7A3FF00F073FF0320FFF79EFF3C
:102A600000F018F9FDF7C6FC034A137B23F00103BD
:102A7000137308BD4A090020F80100202DE98048A1
:102A8000DFF80091A7B089F30888364D364E6B69A0
:102A9000DFF8F4A0354F43F4007300246B61E023AA
:102AA00085F82230EC772C766C76AC766B6A43F442
:102AB000E0236B62FEF7AAFFFEF73AFE4FF0FF330A
:102AC000AB62EB62FFF7A6F8294DFFF715F840F26D
:102AD0000113ADF8243006ABAB60CDE91F4401F023
:102AE0009FFC2046FFF75AFF0120FFF757FF4FF0EA
:102AF000010B00F0D5FC1F4B6E621F4905934FF48C
:102B000080625346CDE9034BCDE901440094304641
:102B100000F08EF8737B804623F004033046737315
:102B200001F05AFD0F23CDE902431449144B4FF431
:102B3000A072CDE904B4CDE90054384600F078F82D
:102B40007B7BEF6023F004037B7305F11803C5E979
:102B500006332C75C5F80490524641463046FEF7C0
:102B6000D1FD00BF00ED00E0F80100207801002059
:102B7000F00800200E4C000060090020800D0020AD
:102B8000512D000000170020492A000070B50E4B9F
:102B90000E4CA34201D3002070BDD3E9030141EAEA
:102BA000000212F003020BD19D685A61AA4201D1C2
:102BB0001C33EEE75E690E60013259610144F5E7AE
:102BC0006FF01500E8E700BF240100202401002079
:102BD000D3B50C4616461F464FF02003EFF3118184
:102BE00083F31188BFF36F8F43695BB123601B6868
:102BF0004361836901338361002081F31188BFF34E
:102C00006F8F11E056EA070203D123606FF00B00CB
:102C1000F3E70246CDE90067083000F083FA18B9FF
:102C2000024B9B685B69236002B0D0BDF0080020B6
:102C30002DE9FF410E9E0673042646730D9E867392
:102C400000F158050F46D61DC0E916550C9A00250F
:102C500026F007062037C0E90655C0E919768560D9
:102C6000C573C56606F1200802920B9A019288444A
:102C70000A9A009242460446FEF70EFD044B656533
:102C80009B6803B11B6F2367404604B0BDE8F08129
:102C9000F00800202DE9F0472A4E2B4D86B0B046B3
:102CA000B54205F1300410D300F0CAF9264CDFF824
:102CB0009CA04FF4004940F2E7360027444521D359
:102CC00006B0BDE8F04700F0ADBA54F8043C0593F7
:102CD00054F8103C049354F8143C039354F8183CF3
:102CE000029354F81C3C019354F8203C009354E99F
:102CF0000A2354E90C01FFF79BFF54F8303C5D6553
:102D00002546CDE7636A5A1C0DD023EAE3733046AB
:102D10003946C9FB0301B94208BFB042256804D156
:102D2000284600F053FB3034C8E74FF47A72002392
:102D3000FDF7E6F902460B4605F11800514600F092
:102D4000F1FCF0E72401002024010020F9450000F7
:102D500008B5094C4FF02002EFF3118382F311887C
:102D6000BFF36F8F01F098FC2062FEF761F8002836
:102D7000F0D1FEF7E3FCEDE7F00800202DE9F34188
:102D8000044616461F464FF02003EFF3118883F3E5
:102D90001188BFF36F8FC368324A6BB18068916846
:102DA000884219D056EA070318D188F31188BFF377
:102DB0006F8F6FF00F000CE0916891F90E10216198
:102DC0000133E3609368A36088F31188BFF36F8FCA
:102DD000002002B0BDE8F0812169F0E790F90E30E3
:102DE00091F90E109942A8BF194621EAE1718B4270
:102DF0002CDD00F009FB0546CDE900671A482246A4
:102E0000414600F08FF90028E3D04FF02003EFF3A4
:102E1000118683F31188BFF36F8F236821699C4269
:102E200007D033B193F90E309942A8BF194621EA71
:102E3000E171A06890F90E30994209D16DB10A484C
:102E4000314600F0EBF86FF00A00C2E70025D3E747
:102E500000F0DAFA0028F2D1F0E786F31188BFF328
:102E60006F8FF0E7F00800204B09002038B5836829
:102E70000446002B36D01E4A9268934235D1DA7B45
:102E8000013ADA73C368012B05D0013BC36000F03F
:102E9000C9F9002038BD4FF02003EFF3118583F30B
:102EA0001188BFF36F8F0169806890F90E309942E5
:102EB00001D000F0A9FA204601F0C0FBA06058B193
:102EC00090F90E2022610022826701F085FB0948FB
:102ED000294600F0A3F8DAE7E06085F31188BFF334
:102EE0006F8FD4E76FF01500D4E74FF0FF30D1E7D4
:102EF000F00800204B09002038B504464FF02003AD
:102F0000EFF3118583F31188BFF36F8F01F096FB08
:102F100048B10022826701F05FFB29460548BDE801
:102F2000384000F07BB8D4E902329A4218BF01332E
:102F3000A360F2E74B09002037B514461D464FF059
:102F40002003EFF3118183F31188BFF36F8F836840
:102F500043B1013B836081F31188BFF36F8F002081
:102F600003B030BD54EA050306D181F31188BFF3E5
:102F70006F8F6FF00F00F3E70246CDE9004502487E
:102F800000F0D0F8ECE700BF4B09002010B5084C6A
:102F900023685BB1FEF71EFA03462068054A034426
:102FA000BDE810401361002101F086BB10BD00BFD9
:102FB00028090020F0080020F8B504460D464FF01F
:102FC0002003EFF3118683F31188BFF36F8F104B4B
:102FD00000224FF4004740F2E73000211A61E7FB7E
:102FE000040100234FF47A72FDF78AF8002C094B94
:102FF00009DC1860084B1D60FFF7C8FF86F31188D5
:10300000BFF36F8FF8BD0228B8BF0220F1E700BF01
:10301000F0080020280900202409002049B9EFF316
:10302000058030B9054B5A6A9B689A4201D0FEF779
:10303000A9BA81F31188BFF36F8F7047F0080020A1
:103040004FF02003EFF3118183F31188BFF36F8FEB
:10305000044B9A68D37B013BD37381F31188BFF390
:103060006F8F7047F008002038B502460C480D4DB0
:1030700001F07BFA044600B9EC68AB684AB95A7BA8
:10308000D20606D1A26922B9DA897F2A01D96B62F8
:1030900038BD9C4201D0FFF779FF6C62F8E700BFB2
:1030A00018090020F008002008B590F90D20437B96
:1030B000002A014604DA03F07F03437301F02DFA7E
:1030C000044B9868431A58425841BDE80840FFF73E
:1030D000CBBF00BFF00800202DE9F04106461446A2
:1030E0001D464FF02003EFF3118783F31188BFF3E0
:1030F0006F8F01F044FA87F31188BFF36F8F6B1C59
:1031000008BFB4F1FF3F08D022462B4606F1180055
:103110000349BDE8F04100F005BBBDE8F08100BF08
:10312000F945000010B5074B9868074B0C4618602E
:103130001146DDE90223FFF7CFFF2046BDE810402E
:10314000FEF720BAF0080020200900202DE9F04108
:1031500005460F4601F0CAFA04464FF02003EFF38C
:10316000118883F31188BFF36F8F124E124BB06832
:103170001860FFF799FFB06810492A463B4618309F
:1031800000F0D0FAB268537B43F01003537340460B
:10319000FEF7F8F901F0AAFA2C44241A4FF00005C2
:1031A00065F10005002C75F10003B8BF002420462E
:1031B000BDE8F081F008002020090020F94500005A
:1031C00070B50446183001F051FA4FF02003EFF3C8
:1031D000118683F31188BFF36F8F94F90D20637B01
:1031E000002A05DA03F07F036373204601F095F9A6
:1031F0000B4D637BA86843F010036373031B5842B5
:103200005841FFF731FF86F31188BFF36F8FAB682A
:10321000A34203D1BDE8704001F09DB970BD00BF6D
:10322000F008002010B54FF02003EFF3118483F372
:103230001188BFF36F8F084B9A68D37B0133D37328
:103240000020FFF711FF84F31188BFF36F8FBDE8F3
:10325000104001F080B900BFF008002070B590F96F
:103260000D20437B002A014604DA03F07F034373F9
:1032700001F053F94B7B174A63F07F0310464B7301
:1032800050F8283FD56A834208BF0023002B38BF7F
:103290000023CBB191F90E6093F90E40A6420FD0F6
:1032A000A41B002C0CDD5868C1E900300160596096
:1032B0009068431A5842BDE870405841FFF7D4BEA9
:1032C000AB4201D01B68E4E7C1E900052960D16287
:1032D000EEE700BFF008002070B501464FF0200374
:1032E000EFF3118483F31188BFF36F8F164B174AE6
:1032F00098681568A8421D4606D1FFF747FE84F37B
:103300001188BFF36F8F70BD00261660104A1268D7
:10331000BAB1C2897F2A14D8427BD20611D10D4A94
:1033200090F90E60126896420BDB0B4A904208D06F
:103330001A698A4202DCFFF791FFDEE7521A1A612E
:10334000DDE700232B61DAE7F008002020090020E8
:1033500028090020240900207801002070B490F989
:103360000D30427B002B2DDBD3062BD183694BBB69
:10337000154962F07F0242730A46CD6A52F8284F1F
:10338000944218BF2346002B38BF0023ABB190F9FD
:103390000E6093F90E40A6420BD0A41B002C08DD52
:1033A0005A68C0E900321060586070BC0020FFF716
:1033B0005BBEAB4201D01B68E8E7C0E9002528608E
:1033C000C862F2E770BC7047F008002010B54FF0FB
:1033D0002002EFF3118482F31188BFF36F8F427BD9
:1033E000510704D484F31188BFF36F8F10BD22F00E
:1033F00004024273FFF7B2FF21460248BDE81040C5
:10340000FFF70CBE4B090020F8B504464FF020032F
:10341000EFF3118683F31188BFF36F8F437BDA06D6
:1034200049B238D18569002D35D103F07F0343734C
:1034300001F073F8437B817363F07F034373174894
:10344000034653F8287F9F4218BF3D46002DC76AA8
:103450001A462B4638BF0023C3B193F90E50A94238
:1034600010D06D1A002D0DDD5A68C4E900321460C9
:103470005C600120FFF7F8FD012086F31188BFF39F
:103480006F8FF8BDBB4201D01B68E5E7C4E9002798
:103490003C60C462EDE7A1730020EEE7F008002075
:1034A000044B002103F12802C3E90A220846FFF772
:1034B00083BD00BFF00800202649F8B58A68264B76
:1034C0009A423DD04FF02003EFF3118583F311882A
:1034D000BFF36F8F8868437B03F07F03437301F072
:1034E0001CF88A68537B084663F07F03537350F8D7
:1034F000283FCE6A834208BF0023002B38BF002339
:10350000CBB192F90E7093F90E40A7420FD0E41B95
:10351000002C0CDD5968C2E900310A605A600120B4
:10352000FFF7A2FD2846BDE8F840FEF72BB8B342EE
:1035300001D01B68E4E7C2E900063260CA62EEE728
:103540004FF02003EFF3118083F31188BFF36F8FE7
:10355000E9E700BFF008002078010020B1F1FF3F4B
:1035600008BFB0F1FF3F08B502460B4606D10B4B32
:103570009868FFF725FE4FF0FF3008BD13430AD1CE
:10358000FFF79AFF00204FF47A7380FB0323D00BE0
:1035900040EA4340F1E7FFF7D9FDF4E7F0080020E7
:1035A000014B9868704700BFF00800202DE9F041FA
:1035B00004464FF02003EFF3118683F31188BFF325
:1035C0006F8F437B1A0705D586F31188BFF36F8F82
:1035D000BDE8F08123F0200242F00801D20920D199
:1035E0004173A36813B1204600F09FFF04F1180057
:1035F00001F03CF804F158074FF00008A56DBD42FA
:1036000000D0B5B90120FFF72FFD104B9B68A342F6
:10361000DAD1EFF30583002BD6D13046FDF7B2FFA8
:10362000D2E703F05F0343F00803437300F075FF34
:10363000D7E7284600F079FF05F1180001F016F8E9
:10364000C5F878802846FFF789FED7E7F008002004
:1036500008B50648064A0749121A00F04DFDBDE8B4
:103660000840054A0549064800F046BD0000002014
:10367000740100204C4C0000000000004C4C000085
:1036800000000020034B1B680BB9FDF7A3BE002010
:10369000704700BF2C09002030B5036868B10A4AA2
:1036A0005268904209D043B1D3E90421D0E90445DE
:1036B000121945EB0101C3E90421426813605A6005
:1036C0000023C0E9003330BD4400002038B5134B5F
:1036D0001C689C4208BF0024FFF7D4FF0546BCB11C
:1036E000D4E90401401B61EBE571012871F100038D
:1036F00011DB6FF000420023824273EB010400DA19
:103700001046074B1B6913B19842A8BF184638BD35
:103710006FF00040F5E70020F3E700BF4400002011
:10372000F0080020B3F1FF3F08BFB2F1FF3F2DE9E1
:10373000F74F044692469B4673D081604FF02003BA
:10374000EFF3118583F31188BFF36F8F6FF00103DF
:10375000B3EB0A084FF0FF3262EB0B09B8F1000F30
:1037600079F100011CDB3048D0E900105B1A62EBF4
:103770000002B3EB0A0662EB0B07012E77F10003A0
:10378000BCBF01260027C4E90467284AD2E9003CEF
:1037900093421ED1C4E9002CCCF8004054602DE0C7
:1037A000FFF770FF1AF1010300934BF1000301933F
:1037B000DDE90023121843EBE073C4E90423E4E7D6
:1037C000B6EB080067EB09016345C4E90401E1D0E9
:1037D0001B68002BDED0D3E90489D4E90467464591
:1037E00077EB0901ECDAB8EB060069EB0701C3E9F6
:1037F00004015968C4E900310C605C6013689342AD
:103800000BD09C4209D1FFF761FF18B1084B1B692F
:10381000834202D00021FDF7ABFD85F31188BFF391
:103820006F8F03B0BDE8F08F7802002044000020C5
:10383000F00800202DE9F74F0646FFF74DFD4FF049
:103840002003EFF3118483F31188BFF36F8F2C4DA6
:10385000DFF8B0A0DFF8B0B02E605146D5F800C058
:10386000DBF800006246D3175845DAE90089CDE954
:1038700000230DD060B1D0E90467B445BB411EDA26
:10388000009BB6EB030C019B67EB0306C0E904C683
:10389000009B13EB0802019B4FF0000643EB09036A
:1038A000C1E900232E60FFF711FF3146FDF760FDEF
:1038B00084F31188BFF36F8F03B0BDE8F08F18EB6E
:1038C00006084FF000024FF0000349EBE679C0E92B
:1038D0000423ACEB0606CAE900892E60FFF7DCFE84
:1038E00084F31188BFF36F8F836898474FF02003EC
:1038F000EFF3118483F31188BFF36F8F0149ADE7B4
:103900002C090020780200204400002010B54FF060
:103910002003EFF3118483F31188BFF36F8FFDF75A
:1039200059FD064BD3E90023121843F1000384F339
:103930001188BFF36F8F1046194610BD7802002022
:10394000024A0349034800F0E7B900BF494C0000B0
:10395000134C0000234C000010B50A4C23681BB127
:1039600001232360002010BD00F0B6F80028F7D036
:103970000138062803D8044B53F8200010BD034833
:1039800010BD00BF30090020A04A0000FE8FFFFFDD
:10399000BFF34F8F0549064BCA6802F4E062134338
:1039A000CB60BFF34F8F00BFFDE700BF00ED00E02D
:1039B0000400FA05F0B4094F094E0A4C0A4A0B4DAF
:1039C0000B494FF0FE333B605268336023600024A4
:1039D0002B60C1F80045F0BC104700BF00B4025096
:1039E00004B4025008B402504C0000200CB4025041
:1039F00000A00250D0E90012014BC3E90012704749
:103A00004C00002048B143682BB1BFF35F8F002307
:103A1000036018467047024870476FF4E0407047F3
:103A2000EA8FFFFF10B5044628B1636813B1002385
:103A30002360636010BD024B02485B689847F4E75F
:103A40004C000020BC4A000010B5044630B1636849
:103A5000002243F001036360226010BD0148FFF7BC
:103A6000A9FFF4E7E44A0000A0B1436883B1012252
:103A7000BFF35B8F50E8003F40E800210029F9D1F7
:103A8000BFF35B8F012BF3D0BFF35F8F0020704734
:103A9000024870476FF4E040704700BFEA8FFFFFB5
:103AA00070B4D0E90065D0E90242094BC3E9024293
:103AB000C3E90065D1E90240D1E90065054B0A6917
:103AC0001A61C3E90065C3E9024070BC704700BFDA
:103AD0005C0000206C00002010B500F033F820B12D
:103AE000032400F067F8204610BD00F035F890B9C7
:103AF00000F0B0F890B90F4B1B681B0EF02B08D1EB
:103B00000D4A0E4B12689A420AD0072400F01CF8A6
:103B1000E7E70624FAE70424204610BD0024F5E771
:103B2000012000F097F804460028F7D1044B1860F4
:103B3000D9E700BF28B9025024BA02500000E020A3
:103B40000CBA02500020704700207047014B1860EB
:103B5000704700BF04BA025010B5114800F048F891
:103B600000B110BD0F4800F043F80028F9D10E4C09
:103B7000204600F03DF80028F3D10C4B0C481C60A7
:103B800000F036F801460028EBD100F02DF804468D
:103B900008B1204610BD00F03FF82046FAE700BF0C
:103BA000A400002098000020A0000020A800002011
:103BB0009C00002008B5084800F024F8074800F0F1
:103BC00021F8074800F01EF8064800F01BF8BDE891
:103BD000084000F00BB800BFA400002098000020AF
:103BE000A00000209C00002000207047704700BF0C
:103BF00008B5034B02681B6810689847002008BD91
:103C00005C00002008B5034B02685B6810689847A9
:103C1000002008BD5C00002070B5094C094D2069EA
:103C2000AB68984718B1084B08485B689847084A42
:103C3000EB68206900211160BDE87040184700BFA3
:103C40006C0000205C0000204C000020084B0000AD
:103C50004409002070B51A4D1A4E0446B26828690E
:103C60009047F0B95CB1184C2368ABB1012B1AD066
:103C7000013B23602869F3689847002070BD124C0F
:103C8000216839B9114B124A0120C3F800051368A5
:103C9000002BFCD101312160F3682869984700208E
:103CA00070BD0C4870BD0A4A1368002BFCD1074A4E
:103CB0006FF07E40C2F80035FFF748FF2368D7E772
:103CC0006C0000205C0000204409002000A002508D
:103CD00010B90250E98FFFFF034658B1426802F065
:103CE0000302012A03D0032A04D1026812B1002082
:103CF000986070476FF0150070474268816002F06D
:103D00000302032A4FF0000203460CBF006810466E
:103D10005A607047002070470FB407B504A951F8E6
:103D2000040B0191FCF77CFB03B05DF804EB04B0DD
:103D30007047038B13F0070305D10368002B0CBFFA
:103D4000002003207047022B05D1438B002B14BFAA
:103D5000002004207047012B05D10368002B0CBF05
:103D6000002005207047002070472DE9F0410D46E6
:103D700007461946281D90461E46FFF7BEFF04461B
:103D800038B13346424629463846A446BDE8F0419C
:103D90006047BDE8F08110B44FF02004EFF31182CA
:103DA00084F31188BFF36F8F416110BC0121FCF7D0
:103DB00045BB10B50C4640B139B1081DFFF78CFF6B
:103DC00028B9A36833F0030301D06FF0150010BDCC
:103DD00038B50C46054658B151B10B6843B14B6834
:103DE00033B11C22002100F0B2F92C61002038BD53
:103DF0006FF01500FBE770B504460E46FFF7D9FFDC
:103E0000051E31DB4FF02003EFF3118183F311889E
:103E1000BFF36F8F638B208B4FF6FF75AB4200F0C3
:103E200007022ED0022A0ED10133638315460123E7
:103E300081F31188BFF36F8FB3B100233146204661
:103E4000FFF793FF10E0830701D0062A0ED100236D
:103E50003360636893B9C4E90066154662B90A46DF
:103E600020460221FCF7EAFA284670BD052A0CBF5D
:103E70006FF085056FF004050023D9E71E606660CA
:103E8000EBE76FF00A05F7E7044608B50846114668
:103E90001A46A047FFF784FBFDF71CFE2DE9F74FFC
:103EA0009946D37814466F2BA3F1410206460F467C
:103EB00001922DD028D8582B14BF0A251025DDF8E3
:103EC0003080AA464FF0000B52465B4630463946DA
:103ED000FCF716F9092AD3B21FD830335F45DBB29D
:103EE00008BF564508F8013D01D3C84512D82378CC
:103EF0009B0605D5082D16D1A37843F00803A370BF
:103F0000404603B0BDE8F08F03F0F703702BD3E712
:103F10000825D4E706460F46D6E7019A192A94BF2A
:103F200037335733DAE7102DEAD1A37843F0100383
:103F3000E5E72DE9F0410746884615461E4614463A
:103F4000B442A4EB050002D33EB923782BB114F898
:103F5000010B4146B8470028F2DABDE8F08170470E
:103F60000022C0E90022826070470269CBB20C21B6
:103F700003FB0121086C00F0070070474FF020039D
:103F8000EFF3118283F31188BFF36F8F036813F08F
:103F9000C00301D08B4207D101230360002082F3CC
:103FA0001188BFF36F8F70474FF0FF30F7E710B500
:103FB0004FF02003EFF3118283F31188BFF36F8F6B
:103FC000036803F00704012C06D10160002082F38E
:103FD0001188BFF36F8F10BD03F0C0038B4214BF75
:103FE0004FF0FF306FF07700F1E74FF02003EFF371
:103FF000118283F31188BFF36F8F036803F0C0034E
:1040000043F00203036082F31188BFF36F8F7047A0
:10401000006910B4CBB21C2403FB0400002110BCC7
:1040200010470020FEF780BB0020FEF7AFBB104614
:10403000FEF762BF38B5CCB20C2305466343006976
:10404000403380211844FFF799FF002805DB696899
:1040500001EBC40463689847002038BD2DE9F8439C
:10406000CDB20C2704696F43064607F1400080215A
:10407000204490469946FFF79AFF002807DB3C440E
:10408000C4E90E89736853F8353098470020BDE8BD
:10409000F8837047704770470020FCF775BE002119
:1040A000012000F000B800F0C5B90146006800F03A
:1040B000C1B908B5FDF75AFBBDE80840FDF7AEBC35
:1040C000034600201A5C02B970470130FAE7034644
:1040D00000201A5C0AB1884200D170470130F8E72D
:1040E000431E013913F8012F11F8010F824201D14B
:1040F000002AF7D1101A7047F0B581EA0004A5072D
:1041000003460BD0013B0A4491421BD1F0BD002A6B
:10411000FCD011F8014B03F8014B013A9C07F6D192
:1041200022F003041D1F96080F19B94205D16FF044
:10413000030505FB06222344E4E751F804CB45F8C8
:1041400004CFF2E711F8014B03F8014FDCE770B53B
:10415000C9B203469C0711D141EA012422F00306AB
:1041600044EA04451E449408B3420DD16FF00305A0
:1041700005FB04221A44934209D170BD002AFCD0E9
:1041800003F8011B013AE5E743F8045BECE703F8A9
:10419000011BF0E74FF0FF307047FEF7CDB984B058
:1041A00004AB03E907009DF80430062B08D14FF05B
:1041B00080430122C3F80025BFF34F8F20BFFDE7E6
:1041C00004B0704784B004AB03E90700002383F315
:1041D0001188BFF36F8F04B070474FF0A0434FF4C6
:1041E0000022C3F808250322C3F84C27002070479B
:1041F00070B50E460168154689B10C68002C38BFB1
:1042000000248A682A4002D04B683046984734B16F
:104210002368002B38BF002321461C46F1E770BD00
:1042200043685B68D3F810350B6000207047436823
:104230005B68D3F8040542400A404240C3F80425B5
:104240000020704743685B680020C3F8081570477A
:1042500043685B680020C3F80C15704743685A68D0
:10426000D2F804354B40C2F804350020704703698A
:10427000586830B558B10024814213D108685CB940
:104280009C685860A14200D198600020086072B913
:10429000002030BD2846EFE720609868814208BFC3
:1042A0009C60F2E705680446002DF3D13AB15A68E4
:1042B0000A60986859600028EAD19960E9E76FF0D0
:1042C0001500E6E72DE9F0410769D0F80480FC68A5
:1042D000D7E90532134324EA0304012600250CB96B
:1042E000BDE8F081264210D0396998F80830E940DD
:1042F00001F00101C1F1030105F01F00C9B240EA5C
:104300004310FDF7A5FD24EA060401357600E6E733
:1043100043681B68D3F80423D10518D5D3F82021AE
:10432000AAB14FF02001EFF3118281F31188BFF39E
:104330006F8FD3F8201131B10021C3F82011D3F8C9
:1043400020110121D96082F31188BFF36F8F426879
:104350005268D20615D54FF02001EFF3118281F398
:104360001188BFF36F8FD3F8581111B10021C3F832
:1043700000154FF48001C3F8081382F31188BFF3CE
:104380006F8F704702690B46D2E9010183E8030091
:104390000020704743681B68D3F88004C3F880048A
:1043A000704742681368D3F8580140B95268120741
:1043B00006D4D3F82001003818BF0120704701202F
:1043C0007047436802691B68D3F8100148B1527CFA
:1043D0000A700020C3F81001D3F8102101221A60DE
:1043E00070474FF0FF30704708B50020FDF75EFCC6
:1043F000FFF7B2BA08B5FCF7FBFFFDF7ADF8BDE873
:104400000840FFF7A9BA004700F074B908B50020CA
:10441000FDF71CF918B9BDE80840FDF707B908BD5C
:104420007047C3681888C0F30800A0F5807358422D
:1044300058417047F8B505460E464FF02003EFF39C
:10444000118783F31188BFF36F8FFFF7A9F8314607
:1044500004462846FFF7C8FF87F31188BFF36F8F24
:104460002046BDE8F840FDF735BB30B50024846137
:1044700041EA020414F00304C0E9023201610CD1E4
:104480004461A34203D1C0E90000002030BD45696A
:104490000D60013441611144F3E76FF01500F5E759
:1044A000F8B504460D464FF02003EFF3118683F371
:1044B0001188BFF36F8F476977B900F0BFF858B123
:1044C0002A684261876700F087F8314604F10800E6
:1044D000BDE8F840FEF7A2BD2B6862691A602B6840
:1044E0006361A369013BA36186F31188BFF36F8FFA
:1044F000F8BDEFF30580003818BF0120704708B5FC
:10450000FCF780FCBDE80840FFF7C4BD034600206F
:10451000C3E90200C3E900337047D0E900321360F9
:104520005A600023C0E90033704708B5FFF7F5FF74
:10453000437B23F0020343730023836008BD0346DB
:1045400020B9EFF305820AB9FDF71CB883F311888F
:10455000BFF36F8F70474FF02003EFF3118083F3A9
:104560001188BFF36F8FFFF7EABF034600688342ED
:1045700003D0002838BF002070470020704738B5AE
:1045800004460D46FEF790FD637B43F00203637320
:10459000B5B12B68A5609D4208BF0023002B38BF32
:1045A00000239BB194F90E1093F90E20914208D08C
:1045B000521A002A05DD5A68C4E9003214605C60B2
:1045C00038BD6A68934201D01B68EAE76B68C4E9AA
:1045D00000531C606C60F3E710B54FF02003EFF35D
:1045E000118483F31188BFF36F8FFEF7B7FE84F356
:1045F0001188BFF36F8F10BD10B501464FF0200337
:10460000EFF3118483F31188BFF36F8F10F80B3C25
:1046100013F0280F0DD151F8103C18380BB1FFF7EB
:1046200084FF11F80B3C23F0140301F80B3CFEF758
:1046300095FE84F31188BFF36F8F10BD38B54FF02E
:104640002003EFF3118583F31188BFF36F8FFFF71A
:104650008CFF044620B1FFF768FF183000F006F821
:1046600085F31188BFF36F8F204638BD10B54FF02A
:104670002002EFF3118482F31188BFF36F8F036878
:104680003BB1FFF709F8002084F31188BFF36F8F67
:1046900010BD6FF01500F7E710B54FF02003EFF3F2
:1046A000118483F31188BFF36F8FFFF70FF884F342
:1046B0001188BFF36F8F10BD70B504460D464FF0E3
:1046C0002003EFF3118683F31188BFF36F8FFEF79A
:1046D000FDFF012805DDA04203DB29462046FCF74B
:1046E00047FE86F31188BFF36F8F70BD08B5FFF7E3
:0E46F0000DF908BD08B1FDF7EFBA704770472D
:0246FE00FFFFBC
:0847000030BAFF7F0100000048
:104708007D1C000000000000DB41000000000000EC
:104718008D2B000000000000F143000000000000A5
:104728009D0F0000AC000020E1230000C400002021
:10473800A90E0000000000001D130000DC0000208E
:10474800611D00000C010020611D0000F400002024
:10475800F543000000000000ED1C00000000000010
:104768001928000007440000000000009F400000D6
:10477800C400002011430000000000009F4000001A
:10478800000000009F400000000000009F40000063
:1047980000000000B1200000000000009F40000061
:1047A800000000009F400000000000009F40000043
:1047B800000000009F400000000000009F40000033
:1047C800000000009F400000000000009F40000023
:1047D800000000009F400000000000009F40000013
:1047E800000000009F40000000000000CD12000003
:1047F800000000009F400000000000009F400000F3
:10480800000000009F400000000000009F400000E2
:10481800000000009F400000000000009F400000D2
:10482800000000009F400000000000009F400000C2
:10483800000000009F400000000000009F400000B2
:10484800000000009F400000000000009F400000A2
:10485800000000009F400000000000009F40000092
:10486800000000009F400000000000009F40000082
:10487800000000009F400000000000009F40000072
:10488800000000009F400000000000009F40000062
:10489800000000009F400000000000009F40000052
:1048A800000000009F400000000000009F40000042
:1048B800000000009F400000000000009F40000032
:1048C800000000009F400000000000009F40000022
:1048D800000000009F400000000000009F40000012
:1048E800FF7FFF7FFF7FFF7FFF7FFF7FFF7FFF7FD0
:1048F800FF7FFF7FFF7FFF7FFF7FFF7FFF7FFF7FC0
:0A490800FF7FFF7FFF7FFF7FFF7F2F
:0E491200FFFFFFFFFFFFFFFFFFFFFFFFFFFFA5
:104920000338FDD870470000DD100000354000005E
:104930005D400000000000006B3F00004D100000D3
:10494000B11000002340000029400000450F000086
:10495000FD0E000000000000000000009940000073
:10496000911400004914000001150000FD1300001F
:104970002000002008000020180000200000000097
:1049800010000020000000200000000000000B06C6
:10499000020000009849000000000000E54B000004
:1049A0002600020700000020ED4B000022000B1142
:1049B0000C0100200E0101000C0100200C00010080
:1049C0000C010020050101000C010020070101007D
:1049D0000C010020010101000C0100200301010075
:1049E0000C01002009010100F40000200801010071
:1049F000F400002006010100F40000201A0101006B
:104A0000F40000200D000000F40000201800000059
:104A10000C0100200A000000F4000020100000003B
:104A2000F40000200E000000F4000020130001003C
:104A3000911D0000214200002F420000454200006D
:104A4000514200005D4200000D1F00006F42000057
:104A500000000000FFFFFFFF00000050000000000A
:104A6000FFFF00000003005001000000C3430000EE
:104A7000DD22000095430000712100008543000005
:104A8000002000400B0000000847000040470000E5
:104A9000484700006847000068470000F5FFFFFF37
:104AA000FF8FFFFFFF8FFFFFFE8FFFFFFE8FFFFFD8
:104AB000FD8FFFFFFC8FFFFFFC8FFFFF6D7574659F
:104AC000785F667265652063616C6C6564207769E8
:104AD0007468204E554C4C20706172616D65746530
:104AE0007200000043616E277420696E6974696109
:104AF0006C697A65206D757465782C2077617320F8
:104B00004E554C4C0D0A0000436F756C64206E6F5F
:104B100074206C6F636B20706F77657220736176A1
:104B200065206D75746578006E7266393136306453
:104B30006B5F6E726635323834300048656C6C6F6E
:104B400020576F726C64212025730A00286E696CEF
:104B500029004661696C656420746F207265626F1C
:104B60006F743A207370696E6E696E6720656E644B
:104B70006C6573736C792E2E2E0A00554152545F6A
:104B80003000434C4F434B007379735F636C6F632A
:104B90006B006D757465785F696E69742063616C14
:104BA0006C65642077697468204E554C4C207061A8
:104BB00072616D6574657200436F756C64206E6F11
:104BC0007420616C6C6F63617465206D75746578B9
:104BD000206265666F726520696E697469616C69CF
:104BE0007A696E6700464C4153485F30005352412A
:104BF0004D5F30004750494F5F31004750494F5F8C
:104C000030000000000001010100000000006D61A3
:104C1000696E0076322E362E302D7263312D6E6322
:104C20007331002A2A2A20426F6F74696E67205AF6
:104C30006570687972204F53206275696C64202515
:0C4C400073202573202A2A2A0A00000095
:104C4C00153D0000010000002401002001000000BF
:104C5C0038010020010000004C0100200100000080
:104C6C0060010020010000009541000000000000E0
:104C7C0000C2010000010300000000000000000061
:104C8C000090D003440000204400002000000000ED
:104C9C00913900003409002001000000493A00005D
:104CAC00253A0000693A0000053A00009000002007
:104CBC00540000208800002000000000800000202C
:104CCC0038090020010000003C0900200100000010
:104CDC004009002001000000700000207C00002032
:0C4CEC00740000206C000020A0000020DC
:104CF800824B00003C49000028490000980200202F
:104D0800AC020020084900007B4B0000804A0000EC
:104D18006C4A0000800800202C000020FE4800009B
:104D2800884B000000000000000000000403002081
:104D380000000000F8480000FB4B0000544A000047
:104D4800304A00004408002048080020F0480000CD
:104D5800F44B0000604A0000304A00004008002080
:084D680064080020E848000087
:104D700024010020240100200000000000000000A9
:104D80000F00000038010020380100200000000062
:104D9000000000000F0000004C0100204C0100202A
:104DA00000000000000000000F0000006001002073
:104DB0006001002000000000000000000F00000063
:04000003000017EDF5
:00000001FF
